:020000040001F9
:10B00000284A002039B5010041B5010043B50100CF
:10B0100045B5010047B5010049B501000000000039
:10B020000000000000000000000000004BB501001F
:10B0300000000000000000004DB501004FB5010008
:10B0400051B5010051B5010065BA010051B50100CB
:10B0500051B5010051B5010049B6010051B50100DB
:10B0600051B5010051B5010051B5010051B50100C4
:10B0700051B5010051B5010051B5010051B50100B4
:10B0800051B50100B1B7010051B5010051B5010042
:10B09000D5B7010051B50100D9B7010051B5010084
:10B0A00051B5010051B5010051B5010051B5010084
:10B0B00051B5010051B50100000000000000000082
:10B0C00051B5010051B5010051B5010051B5010064
:10B0D00051B5010051B50100000000000000000062
:10B0E0000000000000000000000000000000000060
:10B0F0000000000000000000000000000000000050
:10B10000000000000000000000000000000000003F
:10B11000000000000000000000000000000000002F
:10B40000DFF80CD000F0F0F80048004755F40100D8
:10B41000284A0020401E00BF00BF00BF00BF00BF81
:10B4200000BF00BF00BF00BF00BF00BF00BF00BF24
:10B4300000BF00BF00BF00BF00BF00BF00BF00BF14
:10B4400000BF00BF00BF00BF00BF00BF00BF00BF04
:10B4500000BF00BF00BF00BF00BF00BF00BF00BFF4
:10B4600000BF00BF00BF00BF00BF00BF00BF00BFE4
:10B4700000BF00BF00BF00BF00BF00BF00BF00BFD4
:10B4800000BF00BF00BFC5D170470000401E00BF15
:10B4900000BF00BF00BF00BF00BF00BF00BF00BFB4
:10B4A00000BF00BF00BF00BF00BF00BF00BF00BFA4
:10B4B00000BF00BF00BF00BF00BF00BF00BF00BF94
:10B4C00000BF00BF00BF00BF00BF00BF00BF00BF84
:10B4D00000BF00BF00BF00BF00BF00BF00BF00BF74
:10B4E00000BF00BF00BF00BF00BF00BF00BF00BF64
:10B4F00000BF00BF00BF00BF00BF00BF00BFC5D17D
:10B5000070470000056885F308884068FF2464B22E
:10B51000EFF30585002D01D1A646004725460646D6
:10B5200021273FBAF0B40024002500260027F0B4FC
:10B53000F92040B20047000006488047064800470F
:10B54000FEE7FEE7FEE7FEE7FEE7FEE7FEE7FEE7D3
:10B55000FEE7000009B8010001B4010010B5431A6C
:10B56000934209D28318881803E010F8011D03F8EC
:10B57000011D521EF9D210BD40EA01039B0703D002
:10B5800009E008C9121F08C0042AFAD203E011F822
:10B59000013B00F8013B521EF9D210BDD2B201E0CE
:10B5A00000F8012B491EFBD270470022F6E710B5C8
:10B5B00013460A4604461946FFF7F0FF204610BD21
:10B5C000421C10F8011B0029FBD1801A704730B5CE
:10B5D00004460020034600E05B1C934203D2E05C7B
:10B5E000CD5C401BF8D030BD064C074D06E0E0684E
:10B5F00040F0010394E8070098471034AC42F6D3BA
:10B60000FFF702FFA80F0200C80F020030B58C1828
:10B6100010F8012B12F00F0301D110F8013B1209B1
:10B6200006D110F8012B03E010F8015B01F8015B73
:10B630005B1EF9D101E001F8013B521EFBD1A14292
:10B64000E6D3002030BD00002DE9F0470025DFF8EB
:10B65000F090A8464FF4807601242F46304604F03F
:10B660003FF938B1D9F80403204203D0304604F042
:10B670002DF92543361D64007F1CB6B2082FEDD38B
:10B680004FF4BE74204604F02BF938B1204604F084
:10B690001DF92C4845F00045D0F800802A4E15F0E1
:10B6A000FF0F14D0012700242F420CD009EB840196
:10B6B000D1F81005D1F81015C0F3042056F8242055
:10B6C000C1F3014190477F00641C082CECD3002D8E
:10B6D00032DA0024B14609EB04004E4690F95010CE
:10B6E000491C26D090F8507027F0C005284601F07C
:10B6F0008FFF56F82060E6B1BF090120A840A900DD
:10B7000001F1A041D1F8001710EA080FC1F301417F
:10B7100002D0022902D00CE003290AD1032F05D15F
:10B7200002290BD00221284604F0C1F839462846E8
:10B73000B047641C042CCED3BDE8F0870321F2E7A8
:10B740000060004010050050C026002000F01F02DD
:10B75000012191404009800000F1E020C0F88012F2
:10B76000704700F01F02012191404009800000F164
:10B77000E020C0F80011704700F01F020121914045
:10B780004009800000F1E020C0F80012704749072E
:10B79000090E002806DA00F00F0000F1E02080F822
:10B7A000141D704700F1E02080F80014704700007D
:10B7B00007480021C0F84011C0F84411C0F84811F2
:10B7C000C0F84C11C0F80011C0F8041105F064B8BD
:10B7D0000010014004F0FCBF094810B5406848B1B2
:10B7E000804700280AD0BDE81040064A4FF4BB71DC
:10B7F00000F04CBBBDE8104003F0C0BC10BD000021
:10B8000054200020500F0200F0B58C480022041D87
:10B810000378211D081D0126062B17D125782D0739
:10B8200014D10D78C5F30315032D03D1077817F054
:10B83000F00F0ED0042D03D1077817F0F00F08D0C9
:10B84000052D03D1057815F0F00F02D0062B09D095
:10B8500014E04FF08055D5F84452794FC5F3423586
:10B860003D6002E025782D0708D10D78C5F303155A
:10B87000032D03D1057815F0F00F02D0062B06D06A
:10B880001DE0704D2F6827F080772F601AE0257833
:10B890002D0714D10D78C5F30315032D03D10778B7
:10B8A00017F0F00F0ED0042D03D1077817F0F00F2A
:10B8B00008D0052D03D1057815F0F00F02D0062B26
:10B8C0000AD015E04FF08045C5F80C21C5F81021CD
:10B8D0005B4D2D1F2A6002E025782D0708D10D78D9
:10B8E000C5F30315032D03D1057815F0F00F02D031
:10B8F000062B05D066E0524C03236434236002E03B
:10B9000023781B075ED10978C1F30311052959D1AA
:10B91000007810F0F00F55D14B4800684B49086093
:10B920004948001D0068091D086047480830006844
:10B93000091D086044480C300068091D0860424831
:10B9400010300068091D08603F4814300068091D68
:10B9500008603D48183000683C49203108603A488A
:10B960001C300068091D0860374820300068091D38
:10B970000860354824300068091D086032482830C6
:10B980000068091D086030482C300068091D0860F7
:10B990002D48303000682D49403108602A48343045
:10B9A0000068091D0860284838300068091D0860D3
:10B9B00025483C300068091D086023484030006875
:10B9C000091D08601F487438016841F47001016066
:10B9D000BFF34F8FBFF36F8F4FF01021D1F80002EC
:10B9E000002803DBD1F80002002822DA184B1E6081
:10B9F00018480468002CFCD01524C1F800420568E2
:10BA0000002DFCD0C1F8044201680029FCD01A6066
:10BA100001680029FCD0BFF34F8F0A48F038016855
:10BA20000D4A01F4E06111430160BFF34F8F00BF85
:10BA3000FDE70B4909480860F0BD0000E00F00F089
:10BA40003C050040FCED00E00404001020C500406F
:10BA500004E5014000E401400400FA050090D00331
:10BA6000682000200348007F08B105F075B804F095
:10BA7000EFBF00001827002002E008C8121F08C10D
:10BA8000002AFAD170477047002001E001C1121F5F
:10BA9000002AFBD170472DE9FC5F00251688074678
:10BAA0001580406B14468946A8464FF00C0A1123B6
:10BAB0004FF0020B98B101784846032E48D380F826
:10BAC00000B02288521C92B2228083542288521CD9
:10BAD00092B2228009F802102088401C20803A6B24
:10BAE000DAB12088494600F11205B54230D80B542E
:10BAF00020881023401C80B220800B542088401CDA
:10BB000020800F202388155C401ECD54238840B22E
:10BB10005B1C23800028F5DA454697F82E0030B1EB
:10BB200033462246494603F09DFB050011D197F8A4
:10BB30002D0030B132462146484600F011FF050085
:10BB400007D1B87820B32088C846001DB04202D97A
:10BB50005046BDE8FC9F684679DF0028F9D121886E
:10BB6000032008F8010020881921401C80B22080A1
:10BB700008F800102088401C80B2208000EB0801EB
:10BB8000BDF8000005F054F80146208808442080E4
:10BB9000F878B8B1228897F90310D31C4846B3420D
:10BBA000D6D800F802B022880123521C92B222801B
:10BBB00083542288521C92B2228009F802102088F5
:10BBC000401C20807868B8B1218890F90020CB1CF7
:10BBD0004846B342BCD800F801B021880A23491C6A
:10BBE00089B2218043542188491C89B2218009F8F7
:10BBF00001202088401C2080388950B1CDE90046C2
:10BC00004B460622022107F1080005F087F80500DF
:10BC10009FD1388A50B1CDE900464B460722032117
:10BC200007F1100005F07AF8050092D1388B50B179
:10BC3000CDE900464B461522142107F1180005F006
:10BC40006DF8050085D1386A30B133462246494641
:10BC500001F0B2FE0500DBD1786A30B133462246EE
:10BC6000494603F077FC0500D2D197F82C0038B193
:10BC7000334622464946384604F0BCFA0500C7D18F
:10BC8000387838B1334622464946384603F094FCAA
:10BC90000500BDD128465CE710B501220221002035
:10BCA00001F0D0FA08B1072810D1072202210120A3
:10BCB00001F0C8FA08B1072808D100210A22084675
:10BCC00001F0C0FA08B1072800D1002010BD000023
:10BCD00010B598B0382101A8FFF767FC02208DF855
:10BCE000040001248DF8064006208DF8070003208B
:10BCF000ADF814000E48069024210FA8FFF755FC5C
:10BD00004FF496701390B4201490002001460090D8
:10BD10008DF84840074B0FAA01A800F025FB00282A
:10BD200004D0054A40F26A3100F0B0F818B010BDF6
:10BD3000281F002011F90100F0C201000648006828
:10BD40004FF40021044A8143121D1160111D00F4BB
:10BD500000200860704700000405005070B5002402
:10BD6000064D06E06868012110F8340003F0A2FCDB
:10BD7000641C28788442F5D3002070BD1820002070
:10BD8000F8B515460C460646052A01D20720F8BD2F
:10BD900003F072FD18B903F045FD0028F7D11049F2
:10BDA00000204E600C70C1E902500E4D08610DE09C
:10BDB00006EBC4006968009181788DF80110007865
:10BDC000094A694603F0C8FC0028E0D1641EE4B2C9
:10BDD000EED2BDE8F840054A0021024800F0C2B8A2
:10BDE00018200020B40E0200F1EE010081DB0100FA
:10BDF0003EB50446042001901B4802906946204647
:10BE000002F0A6F948B1A0F50041403904D0174A24
:10BE100040F2871100F03AF83EBD13480C38017B20
:10BE2000C90718D04FF6FF720C218088A7DF90B1A8
:10BE3000A0F5405102390ED008280CD0891E0AD036
:10BE4000112808D043F20141884204D0074A4FF438
:10BE5000BD7100F01BF8204602F030F90028DBD05D
:10BE6000024A40F27F11D5E70C1F0020F0C201000A
:10BE700070B5064614460D460C2001F005FA224620
:10BE800029463046BDE8704000F00CB80EB5ADF85C
:10BE90000010CDE901206A46002144F20100FFF7BD
:10BEA000E7FF0EBD08B501238DF800309DF8003086
:10BEB000144B186059609A606FF48041401807D0A5
:10BEC00001280FD1DA60D86800889861D86807E047
:10BED0001A61186980685861186900889861186942
:10BEE0004068D861186858689868D86818695869AF
:10BEF0009869D86972B600BF9DF800000028FBD190
:10BF000062B608BDCC290020014B1B681847000011
:10BF10009C26002038B50C46074BA268097802EB36
:10BF2000420253F82250054A126A0092024604F176
:10BF300008002369A84738BD94290020F41F002079
:10BF4000074910B50A7802EB820201EB8201091D54
:10BF5000FFF7E0FFBDE81040042004F085BA0000C0
:10BF600038270020074B9B6823B12AB120B1006815
:10BF7000037C1BB108207047072070474174426161
:10BF8000002070472C2000202DE9F047804699467C
:10BF900014460F4690074FF0000634D11C4D8CB369
:10BFA00004F06AF80320C5F81490287004F1180012
:10BFB000002107EB4703AC6004EBC102491C16707B
:10BFC00056709770506000EBC3000329F4DBEE60FD
:10BFD0006E70AE701420FFF7B9FB03211420FFF739
:10BFE000D6FB1420FFF7BDFB0A49C1F800800321EE
:10BFF0001120FFF7CCFB0748001F006828610020D4
:10C00000BDE8F08701E00720FAE7AE60FBE700003B
:10C010002C200020081501402DE9F843DFF870902E
:10C020000D461746D9F80810044651B34CB3052DF8
:10C0300002D20720BDE8F883606910B3607C012854
:10C0400021D0002604F034FED9F80810804601EB18
:10C05000C800694604F04EFEB8B1012100F8041B87
:10C060000C4910C0096880E8E200D9F8081001EB1B
:10C07000C8009DF8001041701420FFF77DFB0020E0
:10C08000D8E70820D6E72E46DCE70420D2E70000F8
:10C090002C20002004150140F8B5124E0446B1686A
:10C0A000E1B1DCB16069C8B10027277404F000FE7B
:10C0B0000546B068694600EBC50004F01BFE78B188
:10C0C000022101704460B0689DF8001000EBC500CB
:10C0D00041701420FFF750FB3846F8BD0820F8BD2A
:10C0E0000420F8BD2C20002010B51A4C00224FF47B
:10C0F00080312068FFF790FF20B1174A4FF4097193
:10C10000FFF7C4FE00224FF400416068FFF784FF90
:10C1100020B1114A40F22721FFF7B8FE002242F277
:10C120006661A068FFF778FF20B10B4A40F22A2130
:10C13000FFF7ACFE00224FF42031E068FFF76CFF00
:10C14000002806D0BDE81040034A40F22D21FFF739
:10C150009DBE10BDF80D0200F0C201002DE9F043B4
:10C160000546007D93B00E460024A0B107949DF8CB
:10C170001C0020F00F00401C20F0F00010308DF863
:10C180001C00707B8DF81D009DF81E0020F006003D
:10C19000801C8DF81E001C216846FFF706FA9DF8EA
:10C1A000000040F002008DF80000297D11B140F040
:10C1B000100001E020F010008DF8000001940394BD
:10C1C0000494287D00B107A8CDE9050401278DF866
:10C1D000427042F61920ADF840000D94B07B8DF806
:10C1E0003400F07B8DF835009DF83600142120F0E6
:10C1F0000600801C20F019008DF83600307B8DF889
:10C20000440008A8FFF7D1F90DF140080DF13409F9
:10C21000ADF8287011A8CDE90889ADF82A40ADF82D
:10C220002C700C90A888AB1D08AA6946A2DF0028D4
:10C2300038D1B06898B38DF8427042F60810ADF866
:10C2400040000D94307C8DF834009DF8350020F0CE
:10C25000FF008DF835009DF8360020F00600801CA8
:10C2600020F019008DF836000EA8B16800F0D8FD56
:10C270000646142108A8FFF798F9ADF828600EA823
:10C28000CDE90889ADF82A40ADF82C600C90E8881B
:10C2900005F10E0208A9A3DF002803D101E0FFE7A2
:10C2A000EC81002013B0BDE8F083000010B50E490A
:10C2B0000E4803F092FFC1B20B48683800F04CFA08
:10C2C00000280FD008280DD0A0F54051043909D01E
:10C2D00043F20141884205D0BDE8104004A2A921E3
:10C2E000FFF7D4BD10BD000064230020101F002004
:10C2F0002E2E5C2E2E5C2E2E5C6D61696E2E6300E0
:10C30000F0B50C4693B01F210726ADF80010ADF82C
:10C310000410002750B1C17849070DD56A4602A91B
:10C32000FFF7B9FB002808D102AD02E00025ADF807
:10C3300000706CB1E07810B1304613B0F0BD01AAC6
:10C340000AA92046FFF7A7FB0028F6D10AAA02E0B7
:10C350000022ADF80470BDF80400C3B2BDF80000BF
:10C36000C1B2284672DFE8E770B50D46049916465B
:10C37000040040D0F6B3414800224271C0E90331C5
:10C38000242231463E48FFF7E9F800F0D5F83C4951
:10C390003431A1F1100001602031816038215C3816
:10C3A000FFF703F93648217838380170A178817099
:10C3B000E178C17061784170D4E90412C0E90412D7
:10C3C000D4E90212C0E90212D4E90612C0E9061249
:10C3D000616AD1B100F1AC0100F1B80241628A603A
:10C3E000636A1B880B80616A436A8988998000218F
:10C3F000436A07E0FFE70E2070BD666AB668765CA8
:10C400005654491C9E888E42F7D8A16AD9B11C4A5D
:10C41000AC32A2F10C018A608162A36A9B888B8096
:10C42000A16A836A098819800021836A04E0A66AE8
:10C43000B668765C5654491C9E888E42F7D894F8AC
:10C440002C1080F82C10216A49B10C49143101627A
:10C45000226A52884A80216A026A098811806168CA
:10C4600021B10649891D4160616841602946BDE8E6
:10C47000704003483838FFF743BF0000541F0020C6
:10C480006824002010B502881D4C102A18D0002105
:10C49000112A1BD0192A18D18079002815D160796A
:10C4A000012820D0022824D0032824D004280CD12D
:10C4B0002171E2680846002A07D0BDE81040104705
:10C4C000017D012901D18088208110BD61708088A3
:10C4D00021898842F9D1012006E021690029F4D0A0
:10C4E000BDE810400847022000F04AF80028F4D1C7
:10C4F00010BD0320F8E7032020710420F4E70000BA
:10C50000541F002010B5022801D0032810D1094C77
:10C51000207800280CD000202070607900F030F8DE
:10C52000002805D02169002902D0BDE81040084745
:10C5300010BD0000541F002002480021816181834A
:10C5400081777047541F00200B4810B500780128F0
:10C5500010D10A4C607868B9607910B174DF002896
:10C5600009D101206070607900F00AF810B12169EA
:10C5700001B18847002010BD68240020541F00200E
:10C580002DE9F04F724C87B00026607106A8069620
:10C5900003F0F2FA0127082805D0002871D1069887
:10C5A00010B12770C0E00696FFF7C6FF694D6878A6
:10C5B00010B16079012804D0A87848B160790228C8
:10C5C00006D1E16819B1E7700820884700E0E670FD
:10C5D0006079DFF87C814FF0020A08F118084FF00B
:10C5E000030B012806D1687840B108F1010003F07F
:10C5F00043FA18B16079022802D00AE084F805A055
:10C60000A87820B108F1010003F036FA08B984F8DF
:10C6100005B0287B4FF0040920B96079032801D1C7
:10C6200084F80590287E20B96079042801D16671CC
:10C630002671E16841B16079032801D0042803D153
:10C64000287808B16078C0B1A67018216846FEF756
:10C65000ACFF8DF8006001968DF808600396607954
:10C6600001280FD0022817D03A4E2436A6F15C07D5
:10C6700003281ED004284DD13BE0A770072088472F
:10C68000E3E752E0ADF81260CDF804808DF8007059
:10C69000ADF8106027713FE0CDF804808DF8007090
:10C6A0002889ADF81200A888ADF8100084F804A01D
:10C6B00032E0A88AADF81200288AADF810002548AB
:10C6C000243004F092FB18B1287808B1607810B1DA
:10C6D00084F804B01EE01F488DF808A0039687F880
:10C6E000039000213838FFF70BFE00281DD10520EC
:10C6F0002BE0A88BADF81000288CADF8120015487F
:10C70000243004F072FB18B1287808B1607878B151
:10C7100084F80490607918B1684673DF002804D16A
:10C72000E16809B120798847002007B0BDE8F08FA3
:10C7300008488DF808A0039687F803900021383840
:10C74000FFF7DEFD0028F0D106202071E2E70000AF
:10C75000541F00206824002073B586B0040034D034
:10C76000217C9DF81C20002091422CD00025012620
:10C770000095ADF8006007A8ADF802500190E1887F
:10C78000608A6A46A4DF00281DD19DF81C00207431
:10C79000608AA0F57F41FF3919D0207DB8B102959C
:10C7A000039504950595E088ADF80800BDF80200F2
:10C7B000ADF80C0001988DF80A60CDF810D0059006
:10C7C000608A02A9A6DF08B070BD0E20FBE7082032
:10C7D000F9E738B50D4604001BD0D5B128682060B4
:10C7E0004FF6FF70608228792075FF2020740120A9
:10C7F0008DF8020041F60F00ADF80000221D6946D9
:10C800000120A0DF002803D129462046FFF7A6FC1F
:10C8100038BD0E2038BD08B5002821D000291FD012
:10C820000A88102A17D0112A17D0502A18D1027D51
:10C83000002A15D031F8062F43899A4210D10A8B6D
:10C84000022A0DD10268002A0AD0897E11F0010F58
:10C8500007D0002106E0898801E04FF6FF71418290
:10C8600008BD01218DF800106946904708BD000001
:10C8700070B5054601461C220F48FEF76FFE0F4CAF
:10C8800000262670286830B1016861604068A060A9
:10C89000201D7ADF02E00948001D7BDF00280AD155
:10C8A0004FF6FF7060806670BDE87040044A00215A
:10C8B0000448FFF757BB70BD54250020741F0020AB
:10C8C000510C0200440E020070B5204C0688002571
:10C8D0001D49E289102E15D01D4B112E1ED0122E8F
:10C8E0002BD0502E19D130F8061F914215D1018B53
:10C8F000022912D1807E10F0010F13D0BDE87040E4
:10C9000001F0ACB883884B80D0F81630CB60D0F8FB
:10C910001A0008614D70002AF0D070BD4FF6FF700C
:10C9200048804D701868FFF7B7FB0028F5D0A16963
:10C930000029F2D0BDE87040084750F8062FCA60C1
:10C9400040680861DAE70000741F002054250020C9
:10C95000440E020001480068FFF79EBB440E02002F
:10C960007CB5054608880C460930904201D90C2058
:10C970007CBD684671DF0028FAD121880820685400
:10C9800020881B21401C80B2208029542088401C14
:10C9900080B220802844DDF801100160BDF8051048
:10C9A00081802088801D80B220809DF8001001B118
:10C9B000012129542088401C208000207CBD0000DB
:10C9C00030B585B00D46040039D0BDB36868A8B352
:10C9D0001C4B4FF6FF7020800FCB0DF1040C8CE840
:10C9E0000F0041F23050ADF8000001A8811E63DF56
:10C9F000002821D1221D69460120A0DF00281BD17B
:10CA00009DF80200A071204601F0BAFA002813D167
:10CA1000204601F067FA00280ED12946204601F091
:10CA2000FDFA002808D16868A062A86800B1E06239
:10CA3000054901200870002005B030BDFFE70E2039
:10CA4000FAE70000480E0200881F00203EB50028CB
:10CA50003CD000293AD0826A002A37D00A88102AAE
:10CA600023D0112A33D0502A21D0512A2ED1044666
:10CA70000A4611F8060F022828D14888238A9842CE
:10CA800024D1907A042821D006281FD005281DD053
:10CA90002046891C02F074FF002817D0E16A0029A3
:10CAA00014D003B0BDE830400847898811E0CA8837
:10CAB00003899A420AD108228DF800208A7F20310A
:10CAC0008DF808200191826A694690473EBD4FF675
:10CAD000FF7101803EBD000030B585B028B30388EA
:10CAE000A3F57F44FF3C22D0124B1B78FBB1114BC6
:10CAF00010255B1C00241D7059709A7001250321BC
:10CB0000ADF810100094019402940394018AADF8DA
:10CB1000001004A9CDE902138DF80250ADF80440CD
:10CB200000886946A6DF05B030BD0E20FBE708206F
:10CB3000F9E70000881F00207FB5044601208DF82A
:10CB4000060041F60A00ADF80400454A01A901209B
:10CB5000A0DF00287ED1228804F13C0552B1404874
:10CB60002B46801C009042F62920616800F058FD99
:10CB7000002873D1228952B139482B460A300090DF
:10CB800042F62420E16800F04BFD002866D1228A9D
:10CB900052B133482B461230009042F6252061698D
:10CBA00000F03EFD002859D1228B52B12C482B4673
:10CBB0001A30009042F62720E16900F031FD00288C
:10CBC0004CD1228C52B126482B462230009042F69E
:10CBD0002620616A00F024FD00283FD1228D52B149
:10CBE0001F482B462A30009042F62820E16A00F0C8
:10CBF00017FD002832D1216B71B102A803F098FD16
:10CC000017482B4632300090082202A942F6232012
:10CC100000F006FD002821D1606B58B110492B4669
:10CC20003A3100910279016842F62A2000F0F8FCBE
:10CC3000002813D1A16B81B102A802F05FFF084860
:10CC40002B4642300090072202A942F6502000F005
:10CC5000E7FC00E002E0002800D1002004B070BD35
:10CC6000901F002070B5044601F048FB214616488D
:10CC700000F08AF8144821461838FFF7CCFD20460A
:10CC8000FFF722FE204600F001FA0F4821468030CF
:10CC9000FFF7DCFE20880D4D102802D011280ED1A0
:10CCA0000AE0072000F0F0FA20B1094A4FF4287199
:10CCB000FFF7ECF8A08801E04FF6FF70A88020464F
:10CCC000BDE87040FFF7DEBB14230020001F0020EA
:10CCD000F0C2010030B50446008C8BB0A0F57F4255
:10CCE000FF3A23D005AA204602F0FFF90546ADF829
:10CCF0000000002001900290039004902189ADF87B
:10CD000004100121ADF808008DF8061005A8CDF833
:10CD10000CD00490208C01A9A6DF002804D1BDF816
:10CD20000010A94200D00C200BB030BD0820FBE75A
:10CD300038B5044608682060087960714FF6FF70C6
:10CD40002084002084F82200A4F84C0001208DF8F3
:10CD5000020041F60D000D46ADF80000A21D694627
:10CD60000120A0DF00280ED12946204602F05CF900
:10CD7000002808D1A86828B12946204600F0AAF862
:10CD8000002800D1002038BD08B50A88102A14D028
:10CD9000112A14D0502A15D131F8062F83899A42CE
:10CDA00010D10A8B022A0DD10268002A0AD0897E8E
:10CDB00011F0010F07D0002106E0898801E04FF64D
:10CDC000FF71018408BD01218DF80010694690476C
:10CDD00008BD70B50446B0F84C000D4614280AD1C1
:10CDE00004F126012622881EFEF7B8FBB4F84C0099
:10CDF000401EA4F84C00B4F84C0004EB4001401C69
:10CE0000A4F84C008D8470BD80F82210704770B576
:10CE100004460D460846FEF7D3FB2080656070BDD2
:10CE20000A780270497841700220704700B585B0D9
:10CE3000002348221F49082003F05EFB20B11EA2F8
:10CE400040F2DE21FFF722F86A460121002003F0BC
:10CE50003DFB20B118A24FF43971FFF717F80120FC
:10CE60008DF80C00184803F04DF920B112A240F2E1
:10CE7000EA21FFF70BF8684603F01EFB20B10EA273
:10CE800040F2EE21FFF702F8104803F00BFB20B14F
:10CE900009A240F2F221FEF7F9FF0D4803F044FB2E
:10CEA000002804D004A240F2F621FEF7EFFF05B0FF
:10CEB00000BD0000B42200202E2E5C2E2E5C2E2EF3
:10CEC0005C6D61696E2E6300001E002065CC010060
:10CED0001D070200F0B58FB00D4606461C216846BE
:10CEE000FEF763FB00249DF80000039440F002006D
:10CEF0008DF80000012701948DF8367042F6382035
:10CF0000049405940694ADF834000C94E87B8DF8F5
:10CF10003000287C8DF831009DF83200142120F07B
:10CF20000600801C20F019008DF8320007A8FEF7DB
:10CF30003CFB0DA807900CA8ADF824700890ADF844
:10CF40002640ADF82870A8680B90F08806F1100311
:10CF500007AA6946A2DF0FB0F0BD00001CB5044669
:10CF600081786A460C4802F019FE002813D16078D7
:10CF70000A49C0EBC00001EB80001C231A46694639
:10CF800002F0C8FE054806494C30807A51F820204E
:10CF90002146684690471CBDEC1F0020502600200B
:10CFA0006C0E0200F8B505460820ADF8000001231C
:10CFB0006A461F492846AADF1E4800688047B120FC
:10CFC00044DF18B11C4A8D21FEF760FF11DF18B154
:10CFD000194A9021FEF75AFF4FF01024606913DFC1
:10CFE00018B1154A9321FEF751FF284600F016FFAD
:10CFF00001204FF0E0218205C1F88022D1F80031F4
:10D000005FF0000100FA01F21A420AD04AB202F0BF
:10D010001F0600FA06F55209920002F1E022C2F85A
:10D020008051491C2029EDD3606900F007F8F8BD54
:10D03000202A00204C200020080F0200FEF762BAD0
:10D040007CB5114E0C004FF00005306015D06946DC
:10D05000002000F0B1F8002815D101A9012000F04E
:10D06000ABF800280FD19DF8041009B1022003E0AD
:10D070009DF8001001B10B202070706810B9FEF708
:10D080000BFE054628467CBD4C1F002010B51A4CEF
:10D090000188606810290ED011292BD1401E6060D4
:10D0A00028D1FEF7F9FD002824D02168002921D0DD
:10D0B000BDE810400847D0B900210122084600F021
:10D0C000C1F808B107280FD107220221012000F082
:10D0D000B9F808B1072807D104220221002000F086
:10D0E000B1F820B1072802D0216801B188476068F3
:10D0F000401C606010BD00004C1F002010B50320D4
:10D1000000F032FA08B1062800D1002010BD00005E
:10D110002DE9F04707460024244802E0641C042C53
:10D1200041D250F82420BA42F8D1042C3BD21F48F7
:10D13000DFF87C901F4E0C38A9F1140841B3012987
:10D140000FD002292FD104EB440030444578002D44
:10D1500029D0D8F81010002925D02846BDE8F0477E
:10D16000084704EB4401755C0E44717861B1D8F84E
:10D1700004100F4A01EB81014900133A8068FEF761
:10D180004BFF08B988F80170B17809F80410DEE7A0
:10D190008068FEF781FF04EB4401314419F8040074
:10D1A0008D78A842D3D0BDE8F0870000140E0200AD
:10D1B000481F00200424002004280CD2074A1268CB
:10D1C000074B13F8203001209840904300D00120F5
:10D1D0000870002070470020FAE70000100500509A
:10D1E000140E020010B5042807D0072811D00A2811
:10D1F0001CD1BDE8104003F011B90D4813218088FF
:10D2000076DF082812D0002810D00AA240F20B3195
:10D2100008E0FFF799F9082808D0002806D005A2F1
:10D2200040F21331BDE81040FEF730BE10BD0000E3
:10D23000001F00202E2E5C2E2E5C2E2E5C6D616950
:10D240006E2E630070B50023042810D20D4D00EB44
:10D250004004012A02D101290CD00022094E00EB22
:10D260004000304461B1012906D0022906D00723CD
:10D27000184670BD0D30C2B22A55F9E74270F7E783
:10D280008270F5E704240020044A01460020127A47
:10D29000D20702D0084600F055B87047341F00206E
:10D2A00070B50E462149054600200A61C1E90165B5
:10D2B000A9071BD50024012211462046FFF7C2FF13
:10D2C000641C042C02D20028F5D00FE070B972085B
:10D2D00004211748FEF754FD40B9FEF73FFD28B979
:10D2E0001348144A00211438FEF73CFEE9070AD01F
:10D2F000114A4FF4F01111600F4B00221B1D1A60F0
:10D300000D4A1032116000280FD109480B4A002144
:10D310001C38FEF727FE002807D1BDE870400448FE
:10D320000121074A1838FEF71DBE70BD341F0020CA
:10D33000240E0200A5D5010008050050B9F2010035
:10D340003DBD01002DE9F84F854EDFF810A24FF4E6
:10D35000E01CF16807462CEA010C0091002071687E
:10D360000AF10404251D7F4B4FF400324FF4802B4B
:10D3700001EB810E8146182F16D2DFE807F00C175B
:10D38000173A4E607083868F868FEAA0A0A0A0A077
:10D39000CAD1D8E1EAEA009A4FF4F0119143216032
:10D3A000C5F8009086F80090BDE8F88FC4F800C07A
:10D3B0004846C5F80090DAF800C08CF4F01C5FEA2B
:10D3C0008C3C09D522602860022F02D14FF4E16025
:10D3D00008E04FF47A6005E02A602060022F3CD01C
:10D3E0004FF4C8706422B0FBF2F041433770002262
:10D3F0005EE0C4F800C04846C5F80090DAF800C006
:10D400008CF4F01C5FEA8C3C04D5226028604FF459
:10D410004870E7E72A6020601FE0C4F800C0484673
:10D42000C5F80090DAF800C08CF4F01C5FEA8C3C80
:10D4300002D522602860CCE72A602060D0E7C4F8DB
:10D4400000C04846C5F80090DAF800C08CF4F01C23
:10D450005FEA8C3CDED522602860C820C2E7C4F8B1
:10D4600000C04846C5F80090DAF800C08CF4F01C03
:10D470005FEA8C3C02D52260286001E02A602060CF
:10D48000377014E0C4F800C04DE0DAF800002BEA71
:10D490000002226000F48020286008E0DAF8000032
:10D4A0002BEA0001216000F48020286071460022F0
:10D4B0001868BDE8F84FFEF7AFBD21602EE0984632
:10D4C0005868FEF7E9FDD7F1110100D040B1F168CD
:10D4D00001F4F0112160C5F80090C6F80C9063E7E4
:10D4E0004FF40022F26001290CD9C82011FB00F191
:10D4F0006420B1FBF0F1706800224143D8F80400C9
:10D50000FEF78AFDF16801F4F0112960C4F800907B
:10D510004AE74FF4F0112160C5F80090377043E7F7
:10D520004FF4E01121604946C5F8009006E04FF441
:10D53000D01121604946C5F800905A462A60BCE7E0
:10D540004FF4C01121604946C5F800904FF4C02245
:10D55000F4E74FF4F01129604946AEE704050050A6
:10D56000341F0020080E020070B500210C4D01246C
:10D5700055F82120920002F1A042D2F8006704FA87
:10D5800001F3034000D0032326F4403646EA034368
:10D59000C2F80037491C0429EAD3002070BD0000FE
:10D5A000140E020000780221FFF7B2BD05494FF0CA
:10D5B000FF32082841F8202002D3084480F8482090
:10D5C00070470000C0260020F0B54FF0FF3512B1C3
:10D5D0000023082601E008230C260C4C05E000BFC0
:10D5E00054F823707F1C04D05B1CB342F8D3284648
:10D5F000F0BD26185DB286F8305044F82310002A9A
:10D60000F5D1E11881F84800F1E70000C0260020BC
:10D610000249084490F9300070470000C0260020FD
:10D620002DE9F0438FB01E46DDF8589015460F00E7
:10D63000804604D123A26D210020FEF727FC25B9E6
:10D6400020A26E210020FEF721FC1C216846FDF778
:10D65000ACFF00249DF80000039440F002008DF818
:10D660000000012001948DF836000494059406947E
:10D67000ADF834800C9430788DF8300070788DF8E7
:10D6800031009DF83200142120F00600801C20F0AB
:10D6900019008DF8320007A8FDF787FF0DA8079045
:10D6A0000CA808901748ADF82450ADF82640ADF806
:10D6B00028500B974B4607AA69460088A2DF0FB097
:10D6C000BDE8F0832E2E5C2E2E5C2E2E5C2E2E5C62
:10D6D0002E2E5C2E2E5C636F6D706F6E656E747394
:10D6E0005C626C655C626C655F73657276696365CC
:10D6F000735C626C655F6469735C626C655F6469CE
:10D70000732E6300901F00202DE9F0413A48017804
:10D7100001EB810100EB8104D4E9030600EB400139
:10D720003648241D00EB8100B0F808804589476821
:10D7300002F0BBFAB6FBF0F100FB116080B30020F1
:10D7400008FB05776188A288DFF8B48011448D1941
:10D750000022C8F8102040B102F0A7FA6188884280
:10D7600021D0BD4201D1A088E8B1A06803281AD019
:10D7700002F09BFAA18844463144B1FBF0F200FB71
:10D7800012108008C8F80C0002F08FFAB5FBF0F117
:10D7900000FB115078B10020BD4228D068B126E0CE
:10D7A000FFE70120CCE702F080FAB6FBF0F103209E
:10D7B000C8F814101CE00120EEE7ADB2BEB202F0D2
:10D7C00074FAB6FBF0F702F070FAB5FBF0F087429E
:10D7D00001D1701B09E002F068FA064602F065FA12
:10D7E000B5FBF0F100FB1150301A800820610220D7
:10D7F000BDE8F04102F038BE38270020942900200F
:10D80000F41F00200648017801EB810100EB810044
:10D810000079042801D000F059B8012002F024BE9C
:10D82000382700200A480B4A017801EB810100EB00
:10D830008100C18811620079012805D0032801D038
:10D84000042804D1FFF760BF012002F00DBE70472D
:10D8500038270020F41F002000EB8002054800213B
:10D8600000EB820002220171C180C0E90321416105
:10D8700001817047382700202DE9F041114D069EA7
:10D880006C781E2C1BD02F783C441E2C00D31E3CE1
:10D8900004EB840405EB840420716261D1E900018A
:10D8A000C4E90301E38026816878401C687006485B
:10D8B000007808B9FFF7B6FF0020BDE8F08104202A
:10D8C000FBE7000038270020F41F002010B50E4CA5
:10D8D000207800EB800004EB80010020091DFEF79A
:10D8E00019FB2078FFF7B8FF6078401E6070207841
:10D8F000401CC0B220701E2801D100202070BDE85D
:10D900001040002002F0B0BD382700202DE9F05F64
:10D910002648C168F1B3DFF898B00E688146DBF89D
:10D9200000400769C078E11B21F07F45ED1CB0B9CC
:10D93000DFF880804FF48030C8F84403C8F804034F
:10D940001120FDF703FF1120FDF70BFF4FF0010A37
:10D95000C8F800A02F20FDF799FD89F803A0B54273
:10D9600000D23546124BE8193C3320F07F40186056
:10D97000DBF800105A46091B21F07F41001B20F004
:10D980007F40C91C81420FD9106818602F20FDF715
:10D990007DFD00E004E0BDE8F05F1120FDF7ECBE86
:10D9A000BDE8F05F02F068BBBDE8F09F2C200020CE
:10D9B00004150140001001402DE9F041178806468A
:10D9C000B81D14460D46984202D90C20BDE8F081DE
:10D9D0003188072206290AD34FF4486C4FF6FF73AB
:10D9E000614501D9994202D17088062801D21046BA
:10D9F000ECE7604501D99842F9D1994203D09842A9
:10DA000001D08142F3D80520E85520881221401C1E
:10DA100080B2208029542088401C80B22080411987
:10DA2000308803F005F92188084480B2208041192C
:10DA3000708803F0FDF82188084420800020C5E7A5
:10DA400002A240F24D21FEF721BA00002E2E5C2EDC
:10DA50002E5C2E2E5C6D61696E2E6300F8B5134846
:10DA600001F0CAFB114D0026114C0C3D30B161692B
:10DA7000B9B101208DF80000684611E0287820B186
:10DA8000616971B18DF80060F6E7687858B1A168F6
:10DA9000084800220068FEF7BFFA10B1A16901B181
:10DAA00088472E70F8BD6168F2E70000801F0020F3
:10DAB00054250020440E020070B5094B044608208E
:10DAC0009E7A00250E4208D0A4F57F40FF3802D090
:10DAD0001889A04202D10020156070BD052070BDDC
:10DAE0009026002000EB40020748012100EB820055
:10DAF00081724FF6FF710181FF21C1720021016027
:10DB000081808171704700009026002010B5134C71
:10DB1000207900071ED46069401C6061E06808B18C
:10DB200004200AE001F076FB08B1022005E020693C
:10DB300060B16068C10704D00320BDE8104002F066
:10DB4000E3BD40F0010060600020F6E7BDE8104052
:10DB5000FFF758BEBDE8104002F0CCBDF41F002016
:10DB600006494868020707D4820702D540F0010041
:10DB70004860022002F0C8BD02F0BCBDF41F0020C6
:10DB80002DE9F04100260125144C22E0606822694D
:10DB900000EBC607387805FA00F1114217D08A4326
:10DBA000226101F035FE02463878E36805FA00F19B
:10DBB000194002FA00F3994209D17978012901D07C
:10DBC000012100E0002151407A6802B19047761CA3
:10DBD000F6B220788642D9D3BDE8F0811820002023
:10DBE0002DE9FC410E46044681786A46254801F03D
:10DBF000D5FF002828D16078234F00EB400007EBC9
:10DC00008000807A400621D4022E1FD0012E1FD022
:10DC10001E4DA0781E49C0EBC00001EB800100231F
:10DC20001C226846A847A8B1022E0DD020781649BC
:10DC300000EB40000C3101EB80001649807A51F86E
:10DC40002020214668469047BDE8FC81124DE0E760
:10DC5000124DDEE7022EF7D0607800EB400007EBB4
:10DC60008000817A21F04001817207496078403953
:10DC7000C0EBC00001EB80011C231A466846A84790
:10DC8000D4E70000EC1F0020902600207D06020053
:10DC90008C2500205C0E020041FF010071FE010096
:10DCA0002DE9F04705250F4F90468946064600248A
:10DCB000C4EBC40007EB800036B1072231461030B8
:10DCC000FDF785FC18B106E0018B414503D1002525
:10DCD000C9F8004002E0641C072CE9D32846BDE8DF
:10DCE000F08700008C2500207CB5054681B26A468D
:10DCF000074801F053FF040008D17421684601F081
:10DD000077FF040002D1284601F0C0FE20467CBD0A
:10DD1000EC1F002070B505460C46100004D006A28A
:10DD200040F22531FEF7B2F82078152802D12846B6
:10DD3000FEF75EF8002070BD2E2E5C2E2E5C2E2E7F
:10DD40005C6D61696E2E63001FB58DF80C0001F0EB
:10DD5000B1FF20B11A4A40F23F31FEF797F803A80D
:10DD600000F086FD20B1164A40F24231FEF78EF8EF
:10DD70000020CDF805008DF809009DF805006946E2
:10DD800020F01E0040F001000C3020F020008DF843
:10DD9000050007208DF8060010208DF807000948BF
:10DDA000009001208DF80400074800F0CDFE002807
:10DDB00004D0034A4FF45471FEF768F81FBD000009
:10DDC000F0C2010015DD0100021F002001B5054968
:10DDD000684600F079FA002803D0034ABF21FEF715
:10DDE00055F808BD50200020080F020010B5097832
:10DDF00059B103220121FEF76FFE00280AD0BDE8C9
:10DE00001040054AAD21FEF741B80088BDE810403A
:10DE1000FFF7C8B810BD0000080F020030B58BB086
:10DE200000242949009400F0F7FC002816D101A92C
:10DE3000254800F095FC98B12449234800F07CFD6A
:10DE400018B1234A6C21FEF721F8204800DF002892
:10DE500004D01F4A5FF06F01FEF718F80BB030BD19
:10DE600005981A4D102201692960818AA980807D58
:10DE7000A871E81D0599FDF771FB112205F1180045
:10DE80000199FDF76BFB019850F8121F45F82A1F06
:10DE900041686960008928810C4800DF18B10C4A8C
:10DEA0005E21FDF7F3FF0120009004200890CDF8DB
:10DEB00024D007A90448079400F09EF90028CDD08B
:10DEC000034A6621C8E7000050200020EC2900200A
:10DED000080F020070470000014908607047000009
:10DEE0004C20002030B58FB005461C216846FDF758
:10DEF0005CFB00249DF80000019440F018008DF8B0
:10DF000000000394049405940694A8798DF83600D3
:10DF100041F23150ADF834000C949DF830001421DA
:10DF200020F0FF008DF830009DF8310020F00F0048
:10DF3000401C20F0F00010308DF831009DF83200C8
:10DF400020F00600801C20F0080040F011008DF841
:10DF5000320007A8FDF729FB0DA807900CA8089030
:10DF6000ADF824401720ADF82640ADF828000B94FA
:10DF7000A88805F1100307AA6946A2DF0FB030BDDB
:10DF800030B58FB005461C216846FDF70EFB002416
:10DF90009DF80000019440F004008DF80000039407
:10DFA000049405940694A8798DF8360041F2325015
:10DFB000ADF834000C949DF83000142120F0FF00DF
:10DFC0008DF830009DF8310020F00F00401C20F04B
:10DFD000F00010308DF831009DF8320020F006007E
:10DFE000801C20F0180040F001008DF8320007A8D6
:10DFF000FDF7DBFA0DA807900CA80890ADF82440B7
:10E000001420ADF82640ADF828000B94A88805F13F
:10E01000080307AA6946A2DF0FB030BD70B58EB005
:10E020000E4605461C216846FDF7BFFA00249DF800
:10E030000000019440F002008DF800000394049465
:10E0400005940694A8798DF8360041F23450ADF865
:10E0500034000C949DF83000142120F00F00401C77
:10E0600020F0F00010308DF830009DF8310020F0E5
:10E07000FF008DF831009DF8320020F00600801C72
:10E0800020F0180040F001008DF8320007A8FDF7DD
:10E090008CFA0DA807900CA808900220ADF8240077
:10E0A000ADF82640ADF828000B96A88805F12003AE
:10E0B00007AA6946A2DF0EB070BD00003EB5044657
:10E0C0001F48017848F20800002930D084B3217835
:10E0D00000292CD11B4900250968002927D0A178E7
:10E0E000072929D2184AC1EBC10002EB8000807ECB
:10E0F000FF2821D012486A46103001F04FFD002859
:10E1000015D160230422694602A801F003FE02999A
:10E11000491C0CD0602304220C49684601F010FF12
:10E12000002804D1084AA1781C3A42F821503EBD8B
:10E13000FFE748F20E00FAE748F21000F7E70000A8
:10E14000DC1F00209C2600208C250020580E020099
:10E150003EB50C4625490A7848F208015AB38A1D93
:10E1600018B114B1027832BB01E010463EBD204A1E
:10E17000126802B3817807291FD21E4BC1EBC1027E
:10E1800003EB8202927EFF2A17D01A4AA3681C3A38
:10E19000B3B142F82130817814486A46103001F05A
:10E1A000FDFC0028E2D160230422694602A801F0A8
:10E1B000B1FD48B116E008463EBD48F210003EBD34
:10E1C00052F82110A160E6E70298401C0AD06423AF
:10E1D00010226946A06801F09DFD0028EFD1029948
:10E1E00061603EBD48F240003EBD0000DC1F0020E3
:10E1F0009C2600208C250020FEB505462D480C46A7
:10E20000017848F20800002924D0811D1DB314B301
:10E21000A26802B3297800291CD12749096800297E
:10E2200018D0A978072918D2244BC1EBC10203EBFF
:10E230008202927EFF2A10D06A7803F5827302EB85
:10E24000420203EB8202927A120703D56068042827
:10E2500006D20720FEBD0846FEBD48F21000FEBDF6
:10E260001448174E6A46103001F098FC0028F6D189
:10E2700060230422694602A801F04CFD18B90298F7
:10E28000401C00D00F4E60230422211D6846B04779
:10E290000028E4D1642310226846A16801F050FEF2
:10E2A0000028DCD1054BAA781C3BA16843F822105A
:10E2B000FEBD0000DC1F00209C2600208C250020D5
:10E2C00071FE010041FF01000A4A137848F208027A
:10E2D0006BB1931D19B110B1007840B901E0184637
:10E2E0007047054B1B6813B108700020704710463B
:10E2F00070470000DC1F00209C2600202DE9F04F15
:10E30000054693B0FC48FF240E9400784FF0000AB5
:10E3100000285BD0DFF8E483D8F80000002855D04F
:10E3200001A800F099FA20B1F54A4FF41F61FDF7FA
:10E33000ADFD281D05902A20ADF818000027FF200C
:10E340008DF806008DF804700097EC4C28880C3C82
:10E35000BB4610280FD0A8886A460221FFF7ACFB05
:10E3600048B9009800EB400104EB8101C97A8DF8AF
:10E3700006108DF80500DFF884932888A9F14C0970
:10E38000132109F11C02A2F1E006172875D010DC58
:10E3900010281ED011285ED013286FD0142815D154
:10E3A000009800EB400004EB8000C07AFF287DD08D
:10E3B0009AE0D44B182877D01C2876D0522805D163
:10E3C00098F80A0053F8201001A8884713B0BDE858
:10E3D000F08F4FF6FF766A4601213046FFF76CFB5F
:10E3E0000028F3D10099022201EB410004EB8000E8
:10E3F000827211228DF810208DF80510A9880181F4
:10E40000D5F80610016069898180297B8171687D5A
:10E41000C10708D0B849083101EB50000078FF2847
:10E4200008D00E9006E032460EA9A81DFFF738FC72
:10E4300000280FD100990E9801EB410104EB8101F6
:10E44000C8728A7A42F008028A728DF8060001A822
:10E45000FEF784FD6EE1009800EB400004EB8001C4
:10E46000887A20F002008872010708D500060FD5CF
:10E47000002101A8FFF7B4FB0AE0B9E043E09DF8F2
:10E480000600FF2804D001F001FBFF208DF80600F4
:10E490000099102001EB410104EB810188721220E8
:10E4A0008DF8100046E101E0FAE041E1EA890EA9A9
:10E4B0000020FFF7F5FB78B900990E9801EB4101B8
:10E4C00004EB8101C8728A7A42F008028A728DF8E0
:10E4D000060001A8FEF742FD009800EB400004EBA7
:10E4E0008000C07AFF2804D00098C0EBC00109EB7F
:10E4F000810A00980023C0EBC00006EB8002A888C8
:10E50000514682DF62E700988DF8101000EB400161
:10E5100004EB81018B7A43F004038B72CB7AFF2BDF
:10E5200033D0162100EBC0008DF8101002EB8000F4
:10E530001A210830FDF739F8009800EB400004EB91
:10E540008000817A41F0400180F80A100099CDF8EE
:10E550002CB001EB410204EB820208ABD27ACDF879
:10E5600028B0C2EBC20206EB8202CDE90C2BC1EB54
:10E57000C10209EB8201CDE9081BA88808F1040259
:10E5800000217FDF0028BDD1D4E00DF1380C48F226
:10E5900043020020C0EBC00306EB83039B7EFF2BEE
:10E5A00004D0401C0728F5D31746CFE70A78022A83
:10E5B0000CD0C0EBC00206EB8202FD2393760B6801
:10E5C00013618B8893828979917505E0C0EBC00156
:10E5D00006EB8101FE228A768CF8000000990E98E5
:10E5E00001EB410104EB81018DF80600C872ADE733
:10E5F00098F8091021F0010188F80910DDF800C031
:10E600000CEB4C0304EB8300817A21F0040282724C
:10E6100014218DF81010A97921B1C07AFFF764FB9D
:10E62000AF7987E0E979490739D59DF80610FF29C8
:10E6300035D042F008028272EA7A920707D5C1EB20
:10E64000C10206EB8202957E25F001059576C27A1D
:10E65000FF2A6FD014F82320022A0ED0C1EBC1018B
:10E6600006EB810102680A6182888A828079887556
:10E67000887E20F0020088760DE0CCEBCC0209EB1E
:10E680008200428AC1EBC10006EB80000283817EDA
:10E6900021F001018176012101A8FFF7A1FA49E0EB
:10E6A000A8790121B1EB101F2ED100F00F00012835
:10E6B0002AD1009800EB400104EB8101897A090717
:10E6C00022D500EBC00002EB80001A210830FCF7D5
:10E6D0006CFF16208DF81000009800EB400004EB52
:10E6E0008000817A41F06001817298F8091041F050
:10E6F000020188F8091019E0DC1F00209C26002088
:10E70000BC0E02007C0E0200009800EB400004EBFF
:10E710008000817A41F08001817215208DF810000F
:10E7200098F80A0053F8201001A88847002701E054
:10E730008DF810103A4604A901A8FDF7E5FB9DF8F5
:10E74000100012287FF4DEAE009800EB400104EBCD
:10E750008101897A01293FF4D5AEFFF7C3F935E687
:10E760002DE9F043064629480C4689B0017848F265
:10E77000080000293FD0811DF6B3ECB331780029A1
:10E7800039D1234900250968002934D0B0780728F9
:10E7900038D2204FC0EBC00007EB8000807EFF28FE
:10E7A00030D0E560B07807F58E79C0EBC00007EB9C
:10E7B0008000C4E90405E846A5601448C4E900895E
:10E7C000B17807AA103001F0E9F9002813D11C2311
:10E7D0001A4607A9684601F09DFA00280BD1E560AA
:10E7E000B178C1EBC10107EB8101C4E90415C4F89C
:10E7F0000080C4E9019500E002E009B0BDE8F083C3
:10E800000846F8E748F21000F5E70000DC1F00209A
:10E810009C2600208C25002030B5044611B10878D4
:10E82000A0B902E048F20E0030BD0A48002300689B
:10E8300060B1084AFF200C3A887015890520A5426E
:10E84000F2D14B70D07A8870002030BD48F20800B9
:10E8500030BD00009C26002030B1FF2101704170C6
:10E860008170C1700020704748F20E0070470000B0
:10E870002DE9FF4105003AD02B4800240460447282
:10E8800084722046FFF72EF9274824213038FCF700
:10E890008CFE0026DFF89480FF27304601F0F6F862
:10E8A00008F80670761C072EF7D37420ADF8040024
:10E8B0000720ADF806001E481C4900900831684644
:10E8C00001F07CFA00280FD1184E0120083E30706C
:10E8D000287878B1BDF80400BDF80610484381B22D
:10E8E00006F1100001F084F904B0BDE8F08148F2AF
:10E8F0000E00F9E70F4F00250C48A9B202AA083014
:10E9000001F04CF948B9C5EBC50007EB80000023C6
:10E910001C2202A901F0FEF908B13470E4E76D1C75
:10E92000072DE9D3E0E700009C260020E41F00202B
:10E93000B5E901008C2500201B4A137848F2080233
:10E94000F3B1931D18B111B10378CBB901E01846AA
:10E950007047164B1B689BB1837848F20502FF2B6A
:10E9600010D01348C3EBC30300EB8300837E9B07E7
:10E9700006D402690A60828A8A80807D88710022BA
:10E98000104670474078FF28FAD000EB4003074854
:10E990000C3800EB8300837A9B07F1D502680A608C
:10E9A00082888A808079E9E7DC1F00209C2600208D
:10E9B0008C2500202DE9F04F80465E488FB01E4622
:10E9C0000068189F93468A46002872D0742F70D82A
:10E9D0006846FFF741FF20B1574A40F2A151FDF7C9
:10E9E00055FA00248DF800408DF80440CDE90576F5
:10E9F0002546A9B20DAA514801F0D0F828B908223D
:10EA00000DA94046FCF7E3FDD8B16D1C072DF0D3EE
:10EA10009DF80200FF284CD04FF020094FF0400C29
:10EA200004ADBAF1030F0FD0454A1C27B11AB1FB50
:10EA3000F7F1012307291AD20295BBF1000F0BD081
:10EA400010E08DF80250E3E7742F02D08DF804C077
:10EA500067E08DF8049064E03849834010394968D4
:10EA60000B425BD002F0EAF88DF8049046E03149A1
:10EA70004C39A6EB0108B8FBF7F7DFB101F11C0236
:10EA8000B11A2427B1FBF7F702F1240147B32D4A4D
:10EA90008DF804C0964244D0A1F5907252F820201F
:10EAA000B2423BD10295C97A884227D18DF8014004
:10EAB00024E033E01F488DF804908DF801400C30BD
:10EAC000CDE90A409DF802000295C0EBC00002EBC0
:10EAD0008000089007A806901820079105900DE087
:10EAE00030208DF801408DF804008DF80330887ACD
:10EAF000800703D410462421FCF757FD9DF804003D
:10EB0000BAF1020F12D040F0020000BF8DF80400ED
:10EB10005A4601A968460295FDF7F6F90FB0BDE81F
:10EB2000F08F9DF8040040F00300EFE740F0010093
:10EB3000ECE700009C260020BC0E0200EC1F002029
:10EB40008C250020580E0200174A10B512785AB1D1
:10EB500048F20E0258B151B10B6843B1134A146820
:10EB60003CB148F2040010BD48F2080010BD104648
:10EB700010BD0E4C13602C3CD1F8053023634B7A4A
:10EB800084F834300979917223F0050141F00201D3
:10EB90001172D17921F0040141F00301D1710021FA
:10EBA0000170084610BD0000DC1F00209C260020DC
:10EBB0000E4910B54A788C780023A24212D0521C1C
:10EBC000D2B24A70022A00D14B70084A4B781832F0
:10EBD00052F8232002600869104420F07F40086149
:10EBE000012010BD0360002010BD00002C2000207B
:10EBF000002808D0112801D0FDF7A2B902484168C9
:10EC000041F0080141607047F41F002010B51F4C0F
:10EC1000204621784068012910D002292DD00329EF
:10EC200032D1000725D46069401C606100F0F2FA1F
:10EC3000D8B12078BDE8104001F016BC000718D408
:10EC40001348A28B017801EB810100EB8100C188A0
:10EC5000891A0904090CC18003D0BDE8104001F0F5
:10EC60000FBDBDE81040FEF731BEBDE81040FEF715
:10EC7000C9BDBDE8104000F063BC0648617850F89B
:10EC80002100BDE81040004710BD0000F41F002027
:10EC900038270020A00E020028DFFFF7A9BF29DFD8
:10ECA000FFF7A6BF0EB51CA19DF8080020F00F00CD
:10ECB000401C20F0F00010308DF808000A2202A855
:10ECC0007CDF20B1174A4FF49D71FDF7DFF840F269
:10ECD000413078DF20B1134A40F23D11FDF7D6F8FC
:10ECE0000020009001904FF4A071ADF80400ADF841
:10ECF00000104FF4C8704FF40271ADF80600ADF883
:10ED0000021068467ADF002804D0064A40F2471114
:10ED1000FDF7BCF80EBD00004E6F726469635F487A
:10ED2000524D0000F0C201000020704700207047E3
:10ED3000002070472DE9F0474178DFF8A4900546A0
:10ED400001EBC10209EB8200002401EB410109F152
:10ED5000240A4368274626460AEB810163B191F8ED
:10ED60000AC05FEA0C6807D55FEA4C6C04D459F816
:10ED7000226000F108049FB20889D04633463A4623
:10ED80002146A9DF48F241090B281CD000B14846B2
:10ED9000012E16D168784FF6FF7200EB400008EBA9
:10EDA00080000C210089A7DF00280AD0A0F540517F
:10EDB000023913D0082811D0891E0FD011280DD088
:10EDC0000020BDE8F0876878012300EB400008EBE5
:10EDD00080003A4600892146A9DFDBE74846F0E794
:10EDE0006C26002070B50C46014660780A4D00EB99
:10EDF000C00005EB80003823242200F08BFF0028A0
:10EE000008D1617801EBC10105EB81014A68521C10
:10EE100000D14A6070BD00006C2600202DE9F04151
:10EE200088B0804603271A20ADF81C0048782A4E87
:10EE300000EB400006EB80000D4600893B4607AA28
:10EE40006946AADF28BB6878A6F1240400EBC0005D
:10EE500004EB8000BDF81C2069460830FCF7B7FBC6
:10EE60000028687807D000EBC00004EB80014968F7
:10EE700081B11A4E0FE000EB400106EB8101897A67
:10EE8000890724D400EBC00004EB80002421FCF7A8
:10EE90008CFB1CE0124E44F820706878BDF81C20F2
:10EEA00000EBC00004EB800069464260687800EB2C
:10EEB000C00004EB80000830FCF750FB6878382372
:10EEC00000EBC00004EB800124224046B04708B0AC
:10EED0000020BDE8F08100009026002041FF0100E5
:10EEE00071FE0100FFF726BFFFF77CBFFFF796BF5B
:10EEF0002DE9F041124E07460125BD403068FDF76F
:10EF0000CBF800280DD10F4C2069284207D1384694
:10EF100000F07EFC0028E06805D0284304E0A84308
:10EF20002061BDE8F081A843E060206928432061AA
:10EF3000A1683068BDE8F0410022FDF76DB800001F
:10EF4000B40E02001820002070B51B4C2079000779
:10EF50002DD41A48017801EB810100EB81052E695F
:10EF600000F0A3FEE9882A89761E11443144B1FBE2
:10EF7000F0F02169002549B16169814206D1E5605F
:10EF8000606840F001006060002008E000F042F995
:10EF900010B10220E56002E0206920B10320BDE845
:10EFA000704001F0B1BBBDE87040FEF72BBCBDE87E
:10EFB000704001F09FBB0000F41F002038270020A4
:10EFC00010B51349134801F008F9124C81B2183CEE
:10EFD000A068401CA0600E486038FDF77BFE68B159
:10EFE00008280BD0A0F54051043907D043F2014165
:10EFF000884203D008A2D621FCF748FFA06803216D
:10F00000B0FBF1F201FB120000B10120207010BD35
:10F0100074230020181F00202E2E5C2E2E5C2E2E16
:10F020005C6D61696E2E630070B594B00024054676
:10F0300007949DF81C000E4620F00F00401C20F0A5
:10F04000F00010308DF81C00087B8DF81D009DF835
:10F050001E001C2120F00600801C8DF81E00684652
:10F06000FCF7A3FA9DF80000019440F010008DF821
:10F07000000007A8CDE9044001208DF84E0003945C
:10F0800042F637200694ADF84C000D94707B8DF855
:10F090003400B07B8DF835009DF83600142120F047
:10F0A0000600801C20F0180040F001008DF83600AA
:10F0B00008A8FCF77AFA13A808900DA809900EAAE0
:10F0C0000021284600F011F8ADF828001420ADF812
:10F0D0002C000EA8ADF82A400C90E88805F1080332
:10F0E00008AA6946A2DF14B070BD2DE9F0410446BC
:10F0F00040799046002500B1042594F8220008B11B
:10F1000045F00205CAB2FF2908D9090A88F801208A
:10F1100045F0010588F80210032602E088F8012076
:10F120000226B4F84C0008B145F01005002718E09D
:10F13000B01C14280BD9B4F84C0004EB4701C01BD9
:10F14000420004F124002431FCF708FA0DE004EB3E
:10F15000470108EB0602898C1170090A5170C6B28A
:10F160007F1CB4F84C00B842E2DC34F84C0FC01BF2
:10F17000208088F800503046BDE8F081F8B51C4C7E
:10F180002078002832D0206928B10026E06820B11C
:10F19000002526B112E00126F8E70125F9E76846C7
:10F1A00052DF052805D030B1124AA921FCF76EFEC6
:10F1B00004E0012602E021690098884795B960883B
:10F1C000ADF800006946A06861DF052805D030B1C0
:10F1D000084AC821FCF75AFE04E0012502E0D4E900
:10F1E00002018847002EDAD0002DD2D0F8BD0000F1
:10F1F00054200020500F0200054940880A889042A0
:10F2000004D34988884201D8012070470020704704
:10F21000781F002070B50E48017801EB810100EBEA
:10F220008104256900F041FDE18822896D1E1144A9
:10F230002944B1FBF0F1074842698A4205D301D164
:10F24000006910B14FF0000070BD4FF0010070BDBB
:10F2500038270020F41F0020800701D000207047CD
:10F260000120704730B51488E51C9D4201D90C205F
:10F2700030BD02250D5513881C245B1C9BB21380E6
:10F28000CC5413885B1C9BB21380012807D0022842
:10F2900007D0032807D0042807D0072030BD00205E
:10F2A00004E0012002E0CD5401E00320C85410889E
:10F2B000401C1080002030BD0348017AC90702D0ED
:10F2C0000078FEF73FB87047341F00202DE9F04763
:10F2D000DFF8ACA0DAF80C009AF8004080469AF803
:10F2E0000460DAF80890DAF810703AE009EBC40527
:10F2F0002A7833E002EB42016B68521C03EBC10138
:10F30000AB78D2B2934200D100220B78022B02D00C
:10F31000032B23D11FE0D1F804C00346014603E0CC
:10F32000614503D00B46C969C1B1F9E7B1B18B4260
:10F3300005D1C06918B9134F0126BE600027D1F866
:10F3400000C0C969D96149B10B6863440B6005E02D
:10F350000174C06900E000210028F9D16978914268
:10F36000C8D1641EE4B2C1D2CAE903078AF80460B6
:10F37000404502D00120BDE8F0870020FBE70000F7
:10F380002C200020001001402DE9F04705462F48B1
:10F39000002680460778D0F80C904BE0D8F808009B
:10F3A00000EBC70440E002D02846ED691EE020785B
:10F3B000616800EB4002401CC0B201EBC20120704A
:10F3C000A278904200D126700A784868012A2DD18F
:10F3D000027C5ABB8A684260CA6882600A69C2605D
:10F3E0004969816198F8041001B146604268D8F813
:10F3F0001030DFF85CC0D11A21F07F41614502D2A4
:10F400008268114406E0991A826821F07F418A429D
:10F4100002D9511A016000E0066046600121866051
:10F420000174C66101F01AFA002DBCD12078617810
:10F430008842BCD17F1EFFB2B0D2D8F80C1049452B
:10F4400002D00120BDE8F0870020FBE72C2000203F
:10F45000FFFF7F0088B001F083FA304A40F6CD41CB
:10F460000320FDF71DFF20B12D4A40F27931FCF752
:10F470000DFD69460020FDF7E3FD20B1284A4FF459
:10F480005F71FCF703FD9DF80000022844D00024C2
:10F49000FDF7CCFC2046FEF757FCFFF703FCFCF71A
:10F4A00017FC00F0EBFE00F041FE1C216846FCF763
:10F4B0007CF800204FF42031CDE900014FF4702199
:10F4C000029103218DF80C10164989898DF81000DE
:10F4D0001548059015480690ADF80E106846FDF7E2
:10F4E000C7F920B10E4A4FF41971FCF7CFFCFCF7B5
:10F4F000FBFD0320FDF744F820B10DA240F2A1313D
:10F50000FCF7C4FC40F2873448DF0028FCD0044AF2
:10F510002146FCF7BBFCF7E70124B9E7E5D1010080
:10F52000F0C20100142300204DF9010041DA01006E
:10F530002E2E5C2E2E5C2E2E5C6D61696E2E63006D
:10F540000348416821F008014160007800F08CBF59
:10F55000F41F002070B5144682880E4605462088A8
:10F56000111D0144921C994201D8FE2A01D90C2098
:10F5700070BD521C32542088FF21401C80B2208074
:10F5800031542088401C80B220808119288801F0E5
:10F590004FFB2188084480B22080AA8842B1A96824
:10F5A00041B13044FBF7DAFF2088A9880844208065
:10F5B000002070BD072070BDF8B50E4601781446D6
:10F5C0000546012901D1687830B12088821C9A4211
:10F5D0002DD8012902D006E00720F8BD6978014442
:10F5E000891C994223D8181A801E87B2ADF8007082
:10F5F0002188B01C084469467DDF0028EDD12878B9
:10F60000022805D1BDF80010B94201D809210AE04D
:10F610000821012805D16878B84202D8ADF8000069
:10F6200001E0ADF80070BDF80000FE2801D90C2003
:10F63000F8BD2288401CB0542088401C80B2208035
:10F6400031542088401C2080BDF8001008442080E0
:10F650000020F8BD00207047002070470020704750
:10F6600031B540F2E73404E0401E00902046FBF73D
:10F67000D1FE00980028F7D138BD4907090E0028AF
:10F6800006DA00F00F0202F1E02282F8141D03E016
:10F6900000F1E02282F8001400F01F0201219140E5
:10F6A0004009800000F1E020C0F88012C0F800118D
:10F6B000704700002DE9F0478846814600F006FAC1
:10F6C0000124224E0028484618D0FDF7A1FF3044FF
:10F6D00090F848008009032802D0012806D007E0EE
:10F6E0001B48006804FA09F4204201D1022100E01D
:10F6F00003214846BDE8F04700F0D9B800F0F2F920
:10F70000002820D04846FDF783FF0546114F4FF4EF
:10F71000807007EB850100EB8500D1F8102580B2E1
:10F7200042F00102C1F8102500F0D0F8B8F1000F46
:10F7300009D04846FDF76CFF56F82000002802D09B
:10F74000AC40C7F80443BDE8F0870000C0260020A5
:10F7500010050050006000402DE9FC41DFF8A48056
:10F76000044608EB0400002790F930001346C01748
:10F770000E46401C01D0082740E0F278194620468A
:10F78000FDF722FF0546401C37D0B07848B1A000F5
:10F7900000F1A040D0F8001721F00201C0F80017D6
:10F7A00007E000217378204600910A46019100F09D
:10F7B0006DF8F078C0B11448317800EB8500D0F8CE
:10F7C0001025124B1A40C0F810254FF4F8524FF490
:10F7D000403302EA042203EA01410A43D0F810153B
:10F7E0000A43C0F8102509E008EB0500327810F84C
:10F7F000481F41EA8211017000E004273846BDE845
:10F80000FC810000C026002000600040FFE0FCFFFB
:10F8100003490968C14011F0010000D00120704780
:10F820001005005070B5124D95F8540008B108202D
:10F8300070BD0020411E2A18401CC0B282F8301052
:10F840002028F8D300242046FDF7B0FE641CE4B263
:10F850000C2CF8D303210620FFF70FFF05494FF0CA
:10F860000040C1F80403012085F85400002070BD59
:10F87000C026002000600040034890F85400002893
:10F8800000D0012070470000C026002030B541EABA
:10F890004201DDE9034541EA8301800041EA042198
:10F8A00000F1A04041EA0541C0F8001730BD8000DA
:10F8B00000F5E06000F1A040026822F440320260EE
:10F8C000026842EA0141016070470000034908B53F
:10F8D0000844002101600068009008BD00600040FD
:10F8E00002494058012800D00020704700600040C5
:10F8F0004058002800D001207047D0F80403084089
:10F9000000D0012070474058002800D001207047E7
:10F9100010B568B103280FD10220FDF7B5FC00280F
:10F920000AD0BDE8104005A240F28921FCF7AEBA2A
:10F93000BDE8104000F072BD10BD00002E2E5C2E00
:10F940002E5C2E2E5C6D61696E2E6300007800289F
:10F950000AD106483B21808876DF002804D004A223
:10F9600040F24221FCF792BA70470000001F0020CD
:10F970002E2E5C2E2E5C2E2E5C6D61696E2E630029
:10F98000F0B58BB001274FF0020E05468DF80CE064
:10F990008DF81270C88AADF81400088BADF8160007
:10F9A00001F11A00002608960690ADF820E007A89D
:10F9B000ADF8226009900C46A98A288808AAA5DF1C
:10F9C00018B1E96AC9B1884717E09DF81C0010F02A
:10F9D000010F12D0ADF81060288803A9A8DF002815
:10F9E00012D1A17E04F11B00092943D2DFE801F006
:10F9F000420E1D2326282A402C0040F2FD10ADF8AF
:10FA00001000288803A9A8DF0BB0F0BD8DF80060B6
:10FA10000DE006221DE000BF8DF808700190AA6A73
:10FA20006946284690470020EEE78DF80070228B4B
:10FA3000022AF1D2EDE78DF800E0F0E7032012E0B2
:10FA4000042010E005200EE0208B032805D20322BD
:10FA500008212846FDF740F8D6E7B4F81B00ADF8BA
:10FA6000040018B106208DF80000D8E70720FAE757
:10FA70000920F8E70322ECE70021425C0AB10120EB
:10FA80007047491C0629F8D30020704770B5054619
:10FA9000C0EBC5010C48002600EB81042046C4F8E9
:10FAA0001160A4F815601021FBF77FFDFF20207482
:10FAB000A0764FF6FF702083284601F0BFF8024879
:10FAC0001C3840F8256070BD8C250020044908448E
:10FAD00090F93000082801DB0120704700207047B2
:10FAE000C02600200449084490F93000082801D2BB
:10FAF0000120704700207047C026002070B50D001F
:10FB0000044604D10CA24B210020FCF7BFF924B914
:10FB100009A24C210020FCF7B9F9287820706988E7
:10FB20006170090AA170A988E170090A2171E88849
:10FB30006071000AA07170BD2E2E5C2E2E5C2E2EE0
:10FB40005C2E2E5C2E2E5C2E2E5C636F6D706F6EA5
:10FB5000656E74735C626C655C626C655F73657224
:10FB600076696365735C626C655F6469735C626C23
:10FB7000655F6469732E630006490979490701D4FA
:10FB80000820704720B1044949780160002070477F
:10FB90000E207047F41F00203827002070B5124B4C
:10FBA0001B795B0701D4082070BDB8B1B2B10368FE
:10FBB000022B11D20D4C03EB430554F825605EB1C6
:10FBC000466804EB850004894568408901FB0461AF
:10FBD00000FB0450884203D8072070BD0E2070BD82
:10FBE000C2E90031002070BDF41F002094290020DC
:10FBF000F8B5044623480E460079400701D4082092
:10FC0000F8BD24B32068022831D21F4D00EB40001C
:10FC100055F8201059B305EB8000428941680089EE
:10FC200002FB00116068814221D9FFF715FB80B10A
:10FC3000D4E9000200EB400005EB80004368018935
:10FC4000D51AB5FBF1F701FB175585B903E00E2076
:10FC5000F8BD1020F8BDB6FBF1F501FB156535B90F
:10FC60002EB14089414390191944884201D9072097
:10FC7000F8BD002002460090334621460320FDF7E0
:10FC8000FBFDF8BDF41F00209429002010B54FF0B3
:10FC900010204469601C04D000F007F8B4FBF0F0B9
:10FCA00010BD4FF08050406910BD4FF0805000698A
:10FCB00080B2704770B51448002425460470447023
:10FCC0002846FDF7C9FD6D1C1E2DF9D30F4D6C8024
:10FCD000FFF7DCFFC61EFFF7E8FF46430C49AE60A6
:10FCE00000206C6100EB4002401C41F8224001EB17
:10FCF0008202022814815481F4D32C70AC61042058
:10FD0000EC616860002070BD38270020F41F0020DF
:10FD1000942900202DE9F843804626481F461646C0
:10FD200000790C46400702D40820BDE8F883ECB106
:10FD3000B8F1000F1AD02068022815D21E4D00EB32
:10FD4000400055F8201079B105EB800042894168E8
:10FD5000008902FB00116268914205D926B1B042C8
:10FD600002D3F119814203D90720DEE70E20DCE738
:10FD70004046FFF771FAD0B13846FFF76DFAB0B1DF
:10FD80006068FFF769FA90B160683246C119404671
:10FD9000FBF7E4FB00962068002200EB400043469E
:10FDA00055F8205002212046A8470020BDE710202A
:10FDB000BBE70000F41F0020942900202DE9F0414A
:10FDC000294D04460E462879400702D40820BDE894
:10FDD000F081ECB1E6B12068D0B1FFF766FF0146D3
:10FDE000A088814212D3102810D3E08870B1FFF7A9
:10FDF0004DFF471EFFF759FF4743E288A188A868D7
:10FE000002FB0102974201D3890703D00720DEE7F6
:10FE10000E20DCE76988022924D0C6E90010134AC5
:10FE200001EB410302EB83014860206842F82300A4
:10FE3000A0880881E0884881FFF737FFA188E28821
:10FE4000401E01FB0204FFF730FF94FBF0F4FFF7C4
:10FE50002CFFA96804FB0010A8606888401C68801B
:10FE60000020B4E70420B2E7F41F0020942900200A
:10FE7000F8B504461E481E46154600790F46400751
:10FE800001D40820F8BDDFB1D4B12068022815D212
:10FE9000184900EB400051F820207AB101EB8000B6
:10FEA00042894168008902FB00116268914205D9CC
:10FEB00025B1A84202D3A919814203D90720F8BD70
:10FEC0000E20F8BD3846FFF7C7F978B13046FFF786
:10FED000C3F958B16068FFF7BFF938B12B463A460D
:10FEE000214601200096FDF7C7FCF8BD1020F8BDA3
:10FEF000F41F0020942900201049024608780028A9
:10FF00001AD0042818D0022A14D0032A14D10A794E
:10FF100012070FD48A69521C8A61B2F57A7F06D023
:10FF2000022801D000F0A0BA487800F0EDBB0D2007
:10FF3000FCF706B8FEF76ABE70470000F41F002009
:10FF4000F8B504461E481E46154600790F46400780
:10FF500001D40820F8BDDFB1D4B12068022815D241
:10FF6000184900EB400051F820207AB101EB8000E5
:10FF700042894168008902FB00116268914205D9FB
:10FF800025B1A84202D3A919814203D90720F8BD9F
:10FF90000E20F8BD3846FFF75FF978B13046FFF71D
:10FFA0005BF958B16068FFF757F938B12B463A460C
:10FFB000214604200096FDF75FFCF8BD1020F8BD37
:10FFC000F41F0020942900201A4810B58088A0F55D
:10FFD0007F41FF390FD0132176DF20B116A240F206
:10FFE0009B11FBF753FF0020FDF74EF998B112A2C9
:10FFF00040F29D110DE074DF20B1134A40F253111D
:020000040002F8
:10000000FBF744FF0020FDF73FF920B10E4A4FF403
:10001000AB71FBF73BFFFCF79DFC20B106A24FF450
:10002000D371FBF733FFBDE810404FF4FA70FFF7D0
:1000300017BB0000001F00202E2E5C2E2E5C2E2EE3
:100040005C6D61696E2E6300F0C20100084810B556
:10005000007800280BD006480649203000F0BDF893
:1000600081B20448BDE810407038FCF7B2BE10BD44
:10007000001F00208423002070B5012670044FF07B
:10008000E0210025C1F88001084C4010C4F8480365
:10009000C4F8080366602F20FBF7F8F9A660044C4B
:1000A0002F202561FBF7F2F9E57070BD00100140CB
:1000B0002C20002009480A490022C37DC1F80821EC
:1000C00043B1D1F81815437EC268D154417E491C12
:1000D00041767047D1F818057047000018270020B6
:1000E000002000401FB501228DF8080004488DF85B
:1000F00000200191D0E90012684690471FBD000022
:100100001827002008B502490020009108BD000012
:10011000001F00200348417881F00101417002482E
:10012000FCF772BE001F00201423002070B5154894
:100130000124512164258460C0E90015047301463F
:10014000114800F03FF80F488C2110300026016064
:100150004FF4967141600A218160067301460A4896
:10016000083000F02FF807484FF4FA71203005608E
:10017000C0E9011406730146BDE870400248103022
:1001800000F020B864230020101F002010B5036881
:100190000A6889689C1A8C4202D9591A016010BDFC
:1001A00001210260017110BD10B54B6802688968B9
:1001B0009C1A8C4202D91144016010BD00210360D9
:1001C000017110BD0A7B1AB149680160002102E08B
:1001D0000968016001210171704710B5044600797A
:1001E0000028204602D0FFF7DFFF01E0FFF7CEFF37
:1001F000206810BD2DE9F0410746806A1446884604
:10020000C8B3002531E000BFB96A05EB450001EB3A
:100210008006B088801CFE2802D90C20BDE8F08141
:100220002288401C08F8020020881622401C80B258
:10023000208008F800202088401C80B2208000EB3D
:100240000801308800F0F4FC2188084480B2208046
:10025000B28842B1B16871B14044FBF77FF92088A0
:10026000B188084420806D1CEDB297F82C00A8429C
:10027000CAD80020D2E7FFE70720CFE730B59FB00C
:1002800003208DF8680014216846FBF78EF91AA840
:1002900002909DF80C00002420F00F00401C20F07C
:1002A000F00010308DF80C009DF80D00012520F0B5
:1002B000FF008DF80D009DF80E00009420F0FF0067
:1002C0008DF80E009DF80F008DF8045020F00F00FF
:1002D000401C20F0F00010308DF80F009DF8100049
:1002E000694620F0FF008DF810003F48FCF720FD24
:1002F00020B13EA24FF4E671FBF7C8FD142105A81A
:10030000FBF753F99DF82100059420F00F00401CE5
:1003100020F0F00010308DF821009DF822008DF8BB
:10032000185020F00F00401C20F0F00010308DF825
:1003300022009DF82300079420F0FF008DF8230091
:100340009DF8240005A920F00F00401C20F0F000CB
:1003500010308DF8240064208DF8200022481838D1
:10036000FCF737FA20B121A24FF4EF71FBF78EFDB5
:1003700040210AA8FBF719F920A10AA8FCF747FDBC
:100380009DF8640020F00F00401C20F0F0001030B9
:100390008DF864009DF8650020F0FF008DF8650081
:1003A0000AA8FCF7C9FB20B110A240F2E911FBF743
:1003B0006DFD1748CDE91C040B481B94ADF86C503B
:1003C0001BA98030FCF7FCFA20B108A24FF4FC71A5
:1003D000FBF75CFD0F48FDF77FFD0F488078FDF7C8
:1003E000F5FC1FB030BD0000142300202E2E5C2E23
:1003F0002E5C2E2E5C6D61696E2E63004E6F7264F2
:10040000696353656D69636F6E647563746F7200C1
:10041000EDDD0100C9FF0100001F002010B5002024
:10042000FCF732FF20B10CA240F26F21FBF72EFD4A
:10043000FCF764FE20B108A240F27321FBF726FD11
:100440003CDF002806D0BDE8104003A240F277212F
:10045000FBF71CBD10BD00002E2E5C2E2E5C2E2E38
:100460005C6D61696E2E63000C49087040B1012813
:100470000FD002280FD003280FD14869FEF70CBC1B
:1004800000208861C86106484078002805D0FDF743
:10049000C9B900F0F5B800F051B87047F41F00205A
:1004A0003827002018B10349C860002070470E208B
:1004B00070470000542000201CB5034901910091B1
:1004C000694660DF1CBD0000001F002070B50E46AD
:1004D0000546144614211046FBF767F801202080DA
:1004E0000021216121732672657205B1A07200207E
:1004F00070BDFBF7BDBC000070B509B18C0701D021
:10050000072070BD064C0125A1606280054963602B
:1005100010DF0028F5D1257016202EDF70BD0000F9
:1005200054200020F304020018B1034908610020A0
:1005300070470E2070470000542000202DE9F04144
:10054000164C606820F0010060601548017801EBEE
:10055000810100EB81063569FFF7A7FBB5FBF0F7DA
:100560006761FFF7A2FBF1886D1E2944B1FBF0F033
:100570008742606802D140F0020001E020F00200F2
:1005800060602079E16800F00200084304D0002098
:10059000BDE8F04100F0B8B80220F9E7F41F0020F0
:1005A0003827002001484069FEF776BBF41F002081
:1005B00010B5FFF76BFB441EFFF777FB4443FFF7D3
:1005C00074FB05494A69521E5043CA682146BDE87A
:1005D0001040FEF764BB0000F41F00202DE9F0413D
:1005E0001048017801EB810100EB81042569FFF7D8
:1005F0005CFBE188228911442944B1FBF0F200FB45
:100600001216FFF743FB471EFFF74FFB07FB006186
:10061000E08822891044044A28441269BDE8F04168
:10062000FEF73DBB38270020F41F002010B5FFF770
:100630002DFB441EFFF739FB4443FFF736FBB4FBA9
:10064000F0F0BDE81040FEF727BB000070B5FFF7E3
:100650002CFB8608FFF729FB0749496900FB01F4D9
:10066000FFF714FB451EFFF720FB68433246214687
:10067000BDE87040FEF713BBF41F00200020704758
:1006800070B51448017801EB810100EB8104241D51
:10069000FFF70BFB6188104E884211D2FFF705FB74
:1006A00061880D1AFFF701FB8208A188E068084401
:1006B000216928442944FEF7F2FAFFF7F6FA07E029
:1006C000A288E06810448A082169FEF7E8FA608889
:1006D000F06170BD38270020F41F00200448007925
:1006E000000702D4012000F00FB800F003B80000AA
:1006F000F41F00200348416821F008014160407860
:1007000000F002B8F41F002002494870024951F875
:1007100020000047F41F00208C0E020010B5044694
:10072000FFF7EAFB2046BDE81040FBF7EBBE0000F8
:1007300070B50C00054604D110A233210020FBF750
:10074000A5FB25B90DA234210020FBF79FFB2078E3
:1007500028702088000A68702068000CA870206843
:10076000000EE87020792871207A68712089000ACB
:10077000A871A068000CE87170BD00002E2E5C2EE0
:100780002E5C2E2E5C2E2E5C2E2E5C2E2E5C636F2D
:100790006D706F6E656E74735C626C655C626C65C7
:1007A0005F73657276696365735C626C655F6469CB
:1007B000735C626C655F6469732E63000348007943
:1007C000000701D4FDF71EB8FFF794BFF41F002007
:1007D0002DE9F84F204C00256846D4E903B6FEF712
:1007E000E7F98046FEF772FD0746A946B8F1000F0B
:1007F00025D00023009ACC46E06819E0076801463E
:10080000974202D9BA1A026014E0C1F800C0D1F8C8
:100810000C80D21BC8693B448A46B8F1000F07D050
:10082000F71827F07F47C1E90178CAF81C500D4638
:100830000028E3D1E0602846FEF7A6FD04E0284644
:10084000FEF7A2FD00B917B15846FDF75FF884F82E
:100850000490BDE8F88F00002C2000200D4B10B54F
:10086000D96831B102680C68A24204D8A21A0A60A1
:10087000C161D86010BD0B4603E00B46C969121B6D
:1008800021B10C689442F8D3A41A0C600260C161D3
:10089000D86110BD2C2000202DE9F0411F4DEC68DF
:1008A000002C38D01E48002700682969B846401A35
:1008B00020F07F462068B04218D82246361A0744F6
:1008C000E469107C80B182F810806B694BB1D2E989
:1008D0000501984740B113A240F26111FBF7D6FA27
:1008E00002E0D2E905108847002CE3D16978A878A6
:1008F000814206D1401CC0B2A870022801D185F8FF
:1009000002800648A978183040F82170BDE8F0410F
:100910001420FAF731BFBDE8F08100002C20002040
:10092000041501402E2E5C2E2E5C2E2E5C2E2E5C8D
:100930002E2E5C2E2E5C636F6D706F6E656E747301
:100940005C6C69627261726965735C74696D657211
:100950005C6170705F74696D65722E6300000000E9
:1009600010B500231E4A05211846FBF70DFB20B1E8
:100970001CA240F21111FBF789FA1E4A01211E4800
:10098000FBF7F0FA20B117A240F21711FBF77EFA3D
:1009900019481A4A0121001DFBF7E4FA20B111A2FF
:1009A0004FF48E71FBF772FA1348154A0121083093
:1009B000FBF7D8FA20B10BA240F22111FBF766FA3F
:1009C0000D48104A01210C30FBF7CCFA002806D064
:1009D000BDE8104003A24FF49371FBF757BA10BD66
:1009E000EC2000202E2E5C2E2E5C2E2E5C6D61697C
:1009F0006E2E6300ADC20100F80D0200C1EF0100D0
:100A00004D00020015010200064A0020C2F81C0138
:100A10000548838A8168C95C838A5B1C8382C2F82B
:100A20001C15704700200040182700201FB500212A
:100A30008DF8080005488DF80010826801928175D4
:100A4000D0E90012684690471FBD0000182700201B
:100A50002DE9FF413E4D4FF400712846FEF74DFF52
:100A600001273C4C4FF40178002600B34FF49271FB
:100A70002846FEF73DFFD0B1C5F82461C5F80883CC
:100A8000A07E00B96F6002208DF80000D5F88004C8
:100A9000C5F880040390E07D8DF80800E0680190BF
:100AA000E6752676D4E900126846904724E00421D2
:100AB0002846FEF722FFF8B14FF484712846FEF76E
:100AC00017FFC8B1FFF7F6FAE07D617E884213D1C7
:100AD000227E3AB1607EE168E2752269E2602676A4
:100AE000667607E0A07E00B96F60C5F80883E675FA
:100AF000607EE168FFF7F6FA4FF48E712846FEF744
:100B0000F7FE58B1A18AA07D814202D2FFF77CFF97
:100B100004E0C5F81C6108B1FFF788FF4FF4A2712B
:100B20002846FEF7E5FE00280FD0C5F84461A07EF8
:100B300000B12F60E07D002807D0E675607EE16897
:100B400004B0BDE8F041FFF7CDBABDE8FF81000079
:100B500000200040182700207FB5334C4FF49271DD
:100B60002046FEF7D0FE314D0026B0B1C4F8246116
:100B700002208DF80000D4F88004C4F880040390AB
:100B8000D4F83C058DF80800E8680190EE752E76E3
:100B9000D5E90012684690471FE04FF4887120465F
:100BA000FEF7B1FEC8B1C4F81061D4F83C05E97D88
:100BB000C0B2814211D12A7E5AB1E968D4F800321C
:100BC00023F02003C4F80032EA752A69EA602E7621
:100BD00001E0EE75E968FFF785FA4FF4A27120464F
:100BE000FEF791FE50B1C4F84461E87D30B1EE7576
:100BF000D4F83C05E968C0B2FFF774FA4FF490717D
:100C00002046FEF780FE00280CD0C4F82061A87DA5
:100C1000002807D0D4F84C0504B0C0B2BDE870403D
:100C2000FFF704BF7FBD0000002000401827002010
:100C30000870000A487002207047000001218140BE
:100C4000024842688A43426070470000DC1F00206F
:100C500038B515494888A0F57F42FF3A23D04A7835
:100C6000124C521CD2B24A70237B93420AD3091D04
:100C700075DF002817D0A169002914D001B0BDE8A4
:100C80003040084700254D70217C29B13B2176DF9B
:100C900010B1A16901B188476169002903D08DF8BD
:100CA00000506846884738BD741F00205425002036
:100CB0000F480068C005C00D13D0103840B200289E
:100CC00006DA00F00F0000F1E02090F8140D03E0C8
:100CD00000F1E02090F800044009012803D0032827
:100CE00003D00220704700207047012070470000A9
:100CF00004ED00E042788378521CD2B2934200D1D6
:100D000000220378934201D1002070470A704168A5
:100D1000407800EB400001EBC00070472DE9FC413A
:100D20001646DDE90854CDE900541F4680460222EC
:100D300000F00CF8002807D1CDE900543B46102202
:100D40003146404600F002F8BDE8FC812DE9FC5F29
:100D50000026DDE90C4B994692468E468046278850
:100D6000354630E0D8F80400002200EB85006946E3
:100D70000068019001A865DF002830D19DF80000CF
:100D800050451FD10EB1002100E002212288084405
:100D90001118594522D846B9521C90B2208009F842
:100DA00000E02088401C20800126218801A801EB5A
:100DB0000902694665DF002811D120889DF80010DE
:100DC000084420806D1CB8F80000A842CADC56B167
:100DD0002088C01B401E80B2FF2802D90C20BDE82D
:100DE000FC9F09F807000020F9E7017911B9007BA1
:100DF000002800D0012070476C2000208C200020AB
:100E0000AC200020CC200020C4230020E4230020BC
:100E1000102400200D0000000E0000000F00000054
:100E2000100000000D00030011D101000E000300AE
:100E300011D101000F00030011D1010010000300C7
:100E400011D101003425002023D1BCEA5F7823159D
:100E5000DEEF121200000000FFFFFFFF5DF6010051
:100E60001DEE010031ED0100EDEE010059F601002B
:100E7000E5ED01002DED0100E9EE010055F6010060
:100E800035ED010029ED0100E5EE01002D0602001F
:100E90004D060200A5050200DD050200B1050200B5
:100EA000DD06020061DB01000DDB0100BD07020071
:100EB00049EF0100AC290020030000002E2E5C2E1B
:100EC0002E5C2E2E5C2E2E5C2E2E5C2E2E5C636FE6
:100ED0006D706F6E656E74735C626C655C64657674
:100EE0006963655F6D616E616765725C6465766993
:100EF00063655F6D616E616765725F706572697071
:100F0000686572616C2E63002E2E5C2E2E5C2E2E78
:100F10005C2E2E5C2E2E5C2E2E5C636F6D706F6EC1
:100F2000656E74735C6C69627261726965735C6230
:100F30006F6F746C6F616465725F6466755C646624
:100F4000755F6170705F68616E646C65722E6300BE
:100F50002E2E5C2E2E5C2E2E5C2E2E5C2E2E5C2ECB
:100F60002E5C636F6D706F6E656E74735C736F660D
:100F7000746465766963655C636F6D6D6F6E5C73D9
:100F80006F66746465766963655F68616E646C65DD
:100F9000725C736F66746465766963655F68616EC1
:100FA000646C65722E630000C80F0200001F0020F1
:100FB0006C0100000CB60100E80F02006C2000205C
:100FC000BC29000088BA010042010323FFFF0C2A5C
:100FD0000D1801000F1801000A180103EFFFFF04AC
:080FE0001BD5DE011490D003C3
:040000050001B40141
:00000001FF
